:101800001AC040C03FC03EC03DC03CC03BC08CC2BF
:1018100039C038C037C036C035C034C033C032C01C
:1018200031C030C02DC22EC0C1C02CC02BC02AC0B8
:1018300029C028C06FC211241FBECFEFD4E0DEBF85
:10184000CDBF14BE0FB6F894A89580916000886152
:1018500080936000109260000FBE11E0A0E0B1E044
:10186000EAEDFFE102C005900D92AE30B107D9F765
:1018700021E0AEE0B1E001C01D92A93AB207E1F764
:10188000B3D2A9C3BDCF81E085BF82E085BF0895F3
:1018900081E085BF15BE08958F929F92AF92BF924F
:1018A000CF92DF92EF92FF920F931F93CF93DF932C
:1018B000CDB7DEB7DA950FB6F894DEBF0FBECDBF59
:1018C0007E0181ECE80EF11C8E010F5F1F4FAA24F0
:1018D000BB24A01AB10AD12C470180ECC82EC00E3F
:1018E000D801FD01EA0DFB1DE491ED93CA12F9CF79
:1018F000EFE1DE1207C06EEBC8013AD2F40197AFF8
:1019000086AF06C060ECC80133D2F70191838083B3
:10191000D394F2E0EF0EF11C80ECA80EB11CE0E2D3
:10192000DE12DECF60E4C40123D2D3950FB6F89463
:10193000DEBF0FBECDBFDF91CF911F910F91FF9002
:10194000EF90DF90CF90BF90AF909F908F900895D1
:101950005A984298E1ECF0E0808180688083089595
:101960009C016115710509F1409115015091160115
:10197000809113019091140148175907E9F75A9A79
:10198000429A9091C1009F779093C10010921101EB
:101990003093160120931501620F731F7093140189
:1019A0006093130181E08093C60008951F920F9207
:1019B0000FB60F9211242F933F934F935F936F9322
:1019C0007F938F939F93AF93BF93EF93FF93E09198
:1019D0001501F09116018091130190911401E817FF
:1019E000F90711F483E042C08E179F07D8F41092D4
:1019F0001701AEDF80911201882359F098E088E149
:101A00000FB6F894A895809360000FBE9093600085
:101A1000FFCF10921601109215011092140110922E
:101A200013012FC08081813031F080818B3119F01A
:101A300080818330D1F480911101882379F08081F5
:101A40008093C600809115019091160101969093A4
:101A50001601809315011092110113C08BE1809340
:101A6000C60081E0809311010CC080818093C60084
:101A70008091150190911601019690931601809323
:101A80001501FF91EF91BF91AF919F918F917F9140
:101A90006F915F914F913F912F910F900FBE0F90DB
:101AA0001F9018950F931F93CF93C62FBA01809361
:101AB000180189E0E0EFF0E0A9E1B1E001900D92BA
:101AC0008A95E1F7C09322010C2F10E0CC2321F07E
:101AD000A80183E291E01CD26BE06C0F88E191E0F9
:101AE00047D1F801E85EFE4F83879487B801635FB2
:101AF0007F4F88E191E0CF911F910F9131CFCF932C
:101B0000DF93609117016D3008F4B7C0862F90E025
:101B1000885E9E4FFC013197C081D0E0DC2FCC273E
:101B200031978081C80FD11D625088E191E020D1AA
:101B3000C817D90709F0A1C049E050E069E171E098
:101B400080EF90E0D8D120911801892B29F08FE502
:101B5000820F823008F091C0243AB9F048F4223A5A
:101B600079F0233A09F082C081E08093A80185C012
:101B7000263A09F44EC068F0273A09F44EC076C000
:101B80004CE051E062E081ED75C081E08093A701F7
:101B900068C007B600FE05C040E050E060E085ED9B
:101BA00081DF809117018E3229F040E050E060E043
:101BB00082ED78DF80912301803C28F040E050E006
:101BC00060E082ED6FDF4091230180E2489FA00139
:101BD000112420E030E061E0D901A85EBE4F1C96E0
:101BE0007C911C97F901E40FF51F1D968C9190E0F4
:101BF000982F8827870F911D0C0160935700E89557
:101C000011242E5F3F4F2032310531F785E0FA0174
:101C100025C081E08093120124C007B600FE05C0F4
:101C200040E050E060E085ED3DDF809117018E30AF
:101C300029F040E050E060E082ED34DF8091230144
:101C4000803C28F040E050E060E082ED2BDFE09146
:101C5000230180E2E89FF001112483E08093570084
:101C6000E89540E050E060E084ED04C040E050E0E2
:101C700060E082EDDF91CF9115CFDF91CF91089594
:101C80001F920F920FB60F9211242F933F934F93F1
:101C90005F936F937F938F939F93AF93BF93EF93D4
:101CA000FF93809117018D3810F0109217018091E9
:101CB000C60090911001992319F0109210010FC0E5
:101CC000813019F41092170114C08B3121F481E096
:101CD000809310010EC0833011F411DF0AC090917F
:101CE0001701E92FF0E0E85EFE4F80839F5F90933D
:101CF0001701FF91EF91BF91AF919F918F917F91CC
:101D00006F915F914F913F912F910F900FBE0F9068
:101D10001F9018951F920F920FB60F9211240F90DB
:101D20000FBE0F901F9018951F920F920FB60F9233
:101D300011240F900FBE0F901F901895529A3A9A47
:101D4000589AF8941092C5008CE08093C40082E009
:101D50008093C00088ED8093C10086E08093C2002C
:101D6000F7DD69E080EF90E003D0BAD07894089571
:101D7000CF93AC01FC018FEF9FEF70E09F01241B1C
:101D8000350B26173707A4F42191922728E030E07D
:101D9000DC01AA0FBB1F97FF06C0CD01C1E28C2753
:101DA000C0E19C2701C0CD012150310989F7E6CF60
:101DB000CF910895549A539A689A0895CF93DF93D8
:101DC0001F92CDB7DEB78983F5DF549A5C9A53989A
:101DD000689A89818150823010F4709801C0709A9D
:101DE0000F90DF91CF91089580E88093610083E0A8
:101DF0008093610048DDA2DFDDDF82E0DFDF4CDDC4
:101E0000EEEFF7E1259134912817390721F081E0B1
:101E10008093A701D3DF2FE38DE093E02150804032
:101E20009040E1F700C000008091A7018111FFCF31
:101E3000F89480E0C3DF2CDDE0910E01F0910F01FA
:101E4000099580E090E008958F929F92AF92BF92A3
:101E5000CF92DF92EF92FF92CF93DF93EC016881F4
:101E600079818A819B81611571058105910521F434
:101E700064E279ED8BE597E02DE133EF41E050E04E
:101E800050D049015A019B01AC01A7EAB1E465D0E9
:101E90006B017C01ACEEB4EFA50194016AD0DC01CA
:101EA000CB018C0D9D1DAE1DBF1DB7FF03C001975B
:101EB000A109B04888839983AA83BB839F77DF9168
:101EC000CF91FF90EF90DF90CF90BF90AF909F9019
:101ED0008F900895B9DF089580E091E0B5DF08950F
:101EE000A0E0B0E08093000190930101A093020173
:101EF000B09303010895FB01DC0104C08D910190B2
:101F0000801921F441505040C8F7881B990B08955F
:101F1000FB01DC0102C001900D9241505040D8F706
:101F20000895052E97FB16F400940FD057FD05D0A9
:101F300024D007FC02D046F408C050954095309557
:101F400021953F4F4F4F5F4F089590958095709525
:101F500061957F4F8F4F9F4F089531D0A59F900D72
:101F6000B49F900DA49F800D911D11240895B7FF7B
:101F7000F4CFF3DF821B930B0895A1E21A2EAA1B64
:101F8000BB1BFD010DC0AA1FBB1FEE1FFF1FA21729
:101F9000B307E407F50720F0A21BB30BE40BF50B26
:101FA000661F771F881F991F1A9469F760957095AF
:101FB000809590959B01AC01BD01CF010895A29F32
:101FC000B001B39FC001A39F01D0B29F700D811DCE
:0A1FD0001124911D0895F894FFCF2D
:0E1FDA000100000000000100020000000400F1
:0400000300001800E1
:00000001FF
